:1000000012C02CC02BC070C029C028C027C026C079
:1000100025C025C023C022C021C020C01FC01EC0D3
:100020001DC01CC01BC011241FBECFE5D4E0DEBF25
:10003000CDBF10E0A4E6B0E001C01D92AC3EB10718
:10004000E1F710E0A0E6B0E0EEE2F1E102C00590D9
:100050000D92A436B107D9F7D9D067C8D1CF1F9276
:100060000F920FB60F921124EF92FF920F931F93EE
:100070002F933F934F935F938F939F93E090E5006F
:10008000F090E6000091E7001091E800A8019701C8
:100090002E5F3F4F4F4F5F4F9091EB00892F8A5F4C
:1000A0008093EB008D3748F097579093EB00A801B1
:1000B00097012D5F3F4F4F4F5F4F2093E5003093E7
:1000C000E6004093E7005093E8009F918F915F9185
:1000D0004F913F912F911F910F91FF90EF900F90B3
:1000E0000FBE0F901F9018951F920F920FB60F9290
:1000F00011242F933F934F935F936F938F939F930D
:10010000AF93BF93EF93FF9385B3877D85BB6091DA
:10011000E90057E0A62FB0E0E52FF0E033E0EE0F66
:10012000FF1F3A95E1F7EA0FFB1FEC59FF4F4081A3
:10013000AC9888B3942F91708E7F982B98BBAC9A13
:10014000AC9838B3842F90E095958795282F21702F
:100150003E7F232B28BBAC9AAC9838B395958795F6
:10016000282F21703E7F232B28BBAC9AAC9838B344
:1001700095958795282F21703E7F232B28BBAC9A1D
:10018000AC9838B395958795282F21703E7F232B07
:1001900028BBAC9AAC9838B395958795282F2170D9
:1001A0003E7F232B28BBAC9AAC9828B395958795B6
:1001B00081702E7F822B88BBAC9AAC9888B3441F89
:1001C0004427441F8E7F482B48BBAC9A515008F0FF
:1001D000A3CF85B3962F9862887F982B95BB962FD7
:1001E0009F5F983008F090E09093E900FF91EF91C5
:1001F000BF91AF919F918F916F915F914F913F917F
:100200002F910F900FBE0F901F901895EF92FF92B5
:100210000F931F9312BE83B7836083BF89B781603A
:1002200089BF8BE083BD85B5856085BD85B5886058
:1002300085BD14BC89B7806889BF12BA18BA15BACF
:100240008FEF81BB87BB84BB789420E0EE24E394DE
:10025000FF24FA9414C080E090E0422F50E0FC01AB
:1002600063E0EE0FFF1F6A95E1F7E40FF51FEC590D
:10027000FF4FF08201968830910589F72F5F283073
:1002800050F3E092A4002091E5003091E600409107
:10029000E7005091E8008091E5009091E600A09180
:1002A000E700B091E800821B930BA40BB50B885EAE
:1002B0009340A040B04078F31092A40084E190E015
:1002C0006CED70E040ED57E05DD584E690E084D2BF
:1002D00085E090E061E070E0F7D484E190E068EEC2
:1002E00073E047D482E090E06AE770E04FEF5FEFA1
:1002F00024E630E008EE13E09CD1B1D510E088E7A9
:1003000060E070E046E950E021E030E05ED388E74D
:1003100061E070E046E950E021E030E056D389E743
:1003200060E070E046E950E021E030E04ED389E73C
:1003300061E070E046E950E021E030E046D38AE732
:1003400060E070E046E950E021E030E03ED38AE72B
:1003500061E070E046E950E021E030E036D31F5F15
:100360001A3069F620E077CF75D60895089778F4AB
:1003700077FD0DC06830710554F457FD08C090E05A
:10038000483051050CF091E081E0982701C090E0E1
:10039000892F0895FF920F931F93CF93DF93F82E29
:1003A0008B01EA01E3DF8823A9F0FE0193E0EE0F61
:1003B000FF1F9A95E1F7E00FF11FEC59FF4F2081E5
:1003C00081E090E002C0880F991FFA94E2F78095CF
:1003D00082238083DF91CF911F910F91FF90089529
:1003E000FF920F931F93CF93DF93F82E8B01EA01B7
:1003F000BDDF8823A1F0FE0133E0EE0FFF1F3A9529
:10040000E1F7E00FF11FEC59FF4F208181E090E010
:1004100002C0880F991FFA94E2F7282B2083DF91FE
:10042000CF911F910F91FF900895FF920F931F930B
:10043000CF93DF93F82E8B01EA0198DF882389F0B0
:1004400043E0CC0FDD1F4A95E1F7C00FD11FCC5917
:10045000DF4F888190E002C095958795FA94E2F786
:100460008170DF91CF911F910F91FF9008952130FE
:10047000310511F4B5DF08958DDF089540E050E0B7
:1004800010C0FB01E20FF31FEC59FF4F80832F5F79
:100490003F4F28303105A9F74F5F5F4F4830510576
:1004A00049F020E030E0BA01E3E0660F771FEA95FB
:1004B000E1F7E7CF08950BC020E000000000000046
:1004C0000000000000002F5F2A35B9F70197009760
:1004D00099F708952F923F924F925F926F927F9279
:1004E0009F92AF92BF92CF92DF92EF92FF920F93C3
:1004F0001F93CF93DF93982E5B01CC24DD2447E03C
:10050000242E312C8FEFA8168FEFB80611F4760148
:1005100003C07101EC18FD0800E010E02701089409
:100520004108510837010894611C711C36C08FEFD7
:10053000A8168FEFB80611F4C30101C0C201AC01C7
:100540008AE7981641F4C801BE016FDF282FC80161
:10055000BE01A70117C089E7981649F4C801BA017E
:10056000AE0163DF282FC801B701AE010BC088E7D9
:10057000981651F4CA01BE01A80157DF282FC70100
:10058000BE01A80130E073DF2196C830D10579F6AD
:100590000F5F1F4F0830110519F0C0E0D0E0C7CF42
:1005A0000894C11CD11C88E0C816D10409F0AACF58
:1005B0008FEFA8168FEFB80619F0EE24FF2403C0C2
:1005C00037E0E32EF12C00E010E01EC08AE7981619
:1005D00021F4C801BE01A7010DC089E7981621F4D6
:1005E000C801B701AE0106C088E7981621F4C7011B
:1005F000BE01A801CFDE2196C830D10539F70F5FC3
:100600001F4F0830110519F0C0E0D0E0DFCFDF91B7
:10061000CF911F910F91FF90EF90DF90CF90BF90FF
:10062000AF909F907F906F905F904F903F902F90F2
:1006300008952F923F924F925F926F927F928F9286
:100640009F92AF92BF92CF92DF92EF92FF920F9361
:100650001F93DF93CF93CDB7DEB72E970FB6F894E5
:10066000DEBF0FBECDBF9A8389837C836B835E839D
:100670004D8338872F831A8709874F5F5F4F21F497
:1006800097E0292E312C02C02224332489E0682EE1
:10069000712C89819A81681A790A66DEB30132D495
:1006A0006C0162DEB3012ED47C014424552475C054
:1006B0005BDE8C0159DE9C01C80163E070E022D44E
:1006C00001978C0D9D1D9E878D87181619061CF4A9
:1006D0008615970514F0DE86CD86C90163E070E0CB
:1006E00011D48C01015010400E0D1F1D1016110663
:1006F0001CF4061517050CF087018B816D817E8136
:10070000E9DE8D849E84AA24BB2430C0EB81FC8169
:10071000EA37F10521F4C401B601A10115C08B81AE
:100720009C818937910521F4C401B101A6010CC057
:10073000EB81FC81E837F10541F44D855E854E0D76
:100740005F1DC1016B857C854BDE0894E11CF11CAB
:100750000894C11CD11C89819A81E816F906B4F26B
:100760000894A11CB11C0894811C911CE981FA8198
:10077000AE16BF064CF46801EE24FF24C501800FBD
:10078000911F9C878B87E7CF89859A8594DE089493
:10079000411C511CCD84DE847801EF81F8854E1612
:1007A0005F060CF485CF2E960FB6F894DEBF0FBE11
:1007B000CDBFCF91DF911F910F91FF90EF90DF9010
:1007C000CF90BF90AF909F908F907F906F905F90F1
:1007D0004F903F902F900895AF92BF92CF92DF92AB
:1007E000EF92FF920F931F93CF93DF935C01CC2482
:1007F000DD242AC0B9DD64E070E084D3EC01EE248E
:10080000FF2415C0B1DD8C01AFDD9C01C80168E09B
:1008100070E078D3FC01C90168E070E073D3BC01DB
:10082000CF0147E050E0DCDD0894E11CF11CEC1640
:10083000FD0644F388EE93E03EDE8AE76FEF7FEF3C
:1008400049DE0894C11CD11CCA14DB049CF2DF9160
:10085000CF911F910F91FF90EF90DF90CF90BF90BD
:10086000AF9008957F928F929F92AF92BF92CF9256
:10087000DF92EF92FF920F931F93CF93DF93E82EB7
:10088000F62E742E6901C0E0D0E0F7E08F2E912C97
:10089000E8E0AE2EB12C87E0781661F484010C1BE1
:1008A0001D0BA5014C1B5D0B8E2D90E06F2D70E094
:1008B00071DD09C0AE01415050408E2D90E06F2D8A
:1008C00070E068DD8E018E2D90E06F2D70E0A80144
:1008D00087DDC601F0DD2196C830D105E1F6DF9154
:1008E000CF911F910F91FF90EF90DF90CF90BF902D
:1008F000AF909F908F907F9008954F925F926F92EC
:100900007F929F92AF92BF92CF92DF92EF92FF922F
:100910000F931F93CF93DF93982E162F072F3A0133
:1009200080E0ACDD212F302FC9016C01C0E0D0E0A8
:1009300057E0452E512C34C06114710431F0F5019B
:100940008081A201481B510904C0F7018081482F12
:1009500050E0FAE79F1619F4CE01B8010DC089E7FF
:10096000981621F4CE01BA01A80106C098E799169D
:1009700021F4CA01B801AE0133DD0F5F1F4F0894A7
:10098000A11CB11C0894E11CF11C08301105A1F652
:100990002196E8E0F0E0CE0EDF1EC830D10529F048
:1009A0005601760100E010E0C7CFDF91CF911F9193
:1009B0000F91FF90EF90DF90CF90BF90AF909F90FE
:1009C0007F906F905F904F9008952F923F924F923B
:1009D0005F926F927F928F929F92AF92BF92CF92CF
:1009E000DF92EF92FF920F931F93DF93CF93CDB7D8
:1009F000DEB7C158D0400FB6F894DEBF0FBECDBFF2
:100A0000CF57DF4F8883C158D0402B013A014901AD
:100A100071E4A72EB12CAC0EBD1EF50161E8C62E07
:100A2000D12CCC0EDD1E1192EC15FD05E1F700E096
:100A300010E01E010894211C311C81E088169104ED
:100A4000B9F412C091DC60E470E05CD2E1E4F0E063
:100A5000EC0FFD1FE80FF91F8081882399F70F5FC6
:100A60001F4F91E0908316C0003411055CF312C053
:100A700082E08816910471F4003411055CF4E1E41D
:100A8000F0E0EC0FFD1FE00FF11F80818F5F80838E
:100A90000F5F1F4FF501EE24FF249081892F8150B5
:100AA000863010F49F5F90838081873019F408941A
:100AB000E11CF11C3196EC15FD0579F7D101F5012A
:100AC00080814114510419F097E0981B892F8C9371
:100AD00031961196EC15FD0599F7C301ECDCCF5763
:100AE000DF4F8881C158D040B10140E050E005DFC0
:100AF00082B394E0892782BB80E4E816F10409F010
:100B00009CCFCF57DF4F0FB6F894DEBF0FBECDBFDF
:100B1000CF91DF911F910F91FF90EF90DF90CF90D9
:100B2000BF90AF909F908F907F906F905F904F900D
:100B30003F902F900895AC01DC01FB0120E030E0F4
:100B40009C918081981710F49F5F9C939C91808169
:100B5000891710F491509C932F5F3F4F1196319657
:100B60002034310569F78AE7BA0140E050E0C5DE7C
:100B700008952F923F924F925F926F927F928F9241
:100B80009F92AF92BF92CF92DF92EF92FF920F931C
:100B90001F93DF93CF93CDB7DEB7C058D0400FB6C9
:100BA000F894DEBF0FBECDBF2C017B0100E010E04A
:100BB0005E010894A11CB11C24E0922E91E4C92E80
:100BC000D12CCC0EDD1EF501E00FF11F9082CCDBA5
:100BD000F601E00FF11F68E070E094D180830F5FB1
:100BE0001F4F0034110579F700E010E081E4A82ED2
:100BF000B12CAC0EBD1E6E010894C11CD11C370176
:100C0000C601B5014AE797DFC30155DC0F5F1F4FEF
:100C100008301105A9F75701AA0CBB1CAA0CBB1C74
:100C2000CC24DD24A1E48A2E912C8C0E9D1E1E0165
:100C30000894211C311C2BC000E010E0C101B4015C
:100C40004AE779DFC30137DC0F5F1F4F083011051A
:100C5000A9F7C50130DCEE24FF2486DB8C0184DBA0
:100C60009C01C80160E470E04DD1F401E80FF91F68
:100C7000C90168E070E046D180830894E11CF11C52
:100C800080E2E816F10449F70894C11CD11CC41491
:100C9000D50494F2C058DF4F0FB6F894DEBF0FBEF4
:100CA000CDBFCF91DF911F910F91FF90EF90DF901B
:100CB000CF90BF90AF909F908F907F906F905F90FC
:100CC0004F903F902F9008958F929F92AF92BF9236
:100CD000CF92DF92EF92FF920F931F93CF93DF9308
:100CE0004C018B016130710511F480E001C08FEF80
:100CF000C5DBC0E0D0E038DB68E070E003D1B82E9F
:100D0000A92E32DB68E070E0FDD0D82EC92E2CDB96
:100D100068E070E0F7D0F82EE92E0115110551F4C6
:100D20008B2D9A2D6D2D7C2D4F2D5E2D7EDB8130F0
:100D300011F70CC001301105F1F68B2D9A2D6D2D98
:100D40007C2D4F2D5E2D71DB8823A9F68B2D9A2DDE
:100D50006D2D7C2D4F2D5E2D980189DBC401ABDB01
:100D6000219681E0CF3FD80731F6DF91CF911F91D7
:100D70000F91FF90EF90DF90CF90BF90AF909F903A
:100D80008F9008956F927F928F929F92AF92BF92B1
:100D9000DF92EF92FF920F931F93CF93DF933C016B
:100DA0005B014A0180E06ADB00E010E01CC0DCDA95
:100DB00062E070E0A7D0AC0133E0440F551F3A95D4
:100DC000E1F7481B590BC801BE010ADB2196C83068
:100DD000D10569F70F5F1F4F0830110521F4DD249D
:100DE000EE24FF2429C0C0E0D0E0E1CFBDDAEC0161
:100DF000BBDA68E070E086D0082F8E15E1F0CE01F6
:100E000068E070E07FD0182F8D15A9F090E0602F7A
:100E100070E040E050E009DB882321F0812F602F53
:100E200040E003C0812F602F47E095011BDDC40126
:100E300042DBD12EE02EF3948F2D90E0861597059E
:100E4000ACF2DF91CF911F910F91FF90EF90DF9067
:100E5000BF90AF909F908F907F906F900895EF928A
:100E6000FF920F931F93CF93DF9380E007DB00E0A7
:100E700010E04FEEE42E42E0F42E3AC080E0FEDABD
:100E8000CE0119DB8FEFFADA84E690E014DBCE01B5
:100E900066EF7FEF37D088EE93E034D06F5070402C
:100EA000C60FD71F1C161D064CF388EE93E003DB1C
:100EB000CEEED2E080E0E2DAC7018C1B9D0BFBDABC
:100EC0008FEFDCDA84E690E0F6DACE0166EF7FEFB2
:100ED00019D088EE93E016D06F507040C60FD71F20
:100EE0001C161D063CF30F5F1F4F0230110519F051
:100EF000CEEED2E0C3CFDF91CF911F910F91FF9043
:100F0000EF90089597FB092E07260AD077FD04D0AD
:100F10000CD006D000201AF4709561957F4F08958B
:100F2000F6F7909581959F4F0895AA1BBB1B51E141
:100F300007C0AA1FBB1FA617B70710F0A61BB70B49
:100F4000881F991F5A95A9F780959095BC01CD01EE
:100F500008952F923F924F925F926F927F928F925D
:100F60009F92AF92BF92CF92DF92EF92FF920F9338
:100F70001F93CF93DF93CDB7DEB7CA1BDB0B0FB642
:100F8000F894DEBF0FBECDBF09942A8839884888FF
:100F90005F846E847D848C849B84AA84B984C88495
:100FA000DF80EE80FD800C811B81AA81B981CE0F8C
:100FB000D11D0FB6F894DEBF0FBECDBFED01089571
:100FC000A0E0B0E0E5EEF7E0CCCFEC01A880B9807E
:100FD000CA80DB80A114B104C104D10441F484E2CD
:100FE000A82E89EDB82E8BE5C82E87E0D82EC60135
:100FF000B5012DE133EF41E050E05AD027EA31E46A
:1010000040E050E036D07B018C01C601B5012DE1F6
:1010100033EF41E050E04CD0CA01B9012CEE34EF7F
:101020004FEF5FEF26D06E0D7F1D801F911F97FF42
:1010300004C06150704080409048688379838A83FF
:101040009B839B013F77C901CDB7DEB7EAE0A5CF0F
:10105000B7DF089580E690E0B3DF0895A0E0B0E048
:101060008093600090936100A0936200B09363004E
:101070000895629FD001739FF001829FE00DF11DE2
:10108000649FE00DF11D929FF00D839FF00D749F02
:10109000F00D659FF00D9927729FB00DE11DF91FAE
:1010A000639FB00DE11DF91FBD01CF01112408950B
:1010B00097FB092E05260ED057FD04D014D00AD078
:1010C000001C38F450954095309521953F4F4F4F77
:1010D0005F4F0895F6F790958095709561957F4FD5
:1010E0008F4F9F4F0895A1E21A2EAA1BBB1BFD0133
:1010F0000DC0AA1FBB1FEE1FFF1FA217B307E407F7
:10110000F50720F0A21BB30BE40BF50B661F771F4E
:10111000881F991F1A9469F760957095809590952E
:0E1120009B01AC01BD01CF010895F894FFCFF3
:04112E0001000000BC
:00000001FF
